:02000000DF2BF4
:020008000029CD
:02000E00820767
:10001000443453344334203432342E343034303486
:10002000323432342F34303433342F3430343834A3
:100030004E346534783474342034533465346C343D
:100040005234653476342034443465346334203497
:10005000523465347634203452342F3441342034D1
:100060002034423472346934673468347434203450
:1000700043346F346E347434723461347334743492
:10008000533479347334523465347334653474348E
:10009000443465346634613475346C347434733488
:1000A00045347834693474344D3465346E34753481
:1000B0005234653476342034203453346534743407
:1000C000523465347634443420344F3466346634E4
:1000D000523465347634443420344F346E34203412
:1000E000523465347634523420344F3466346634B6
:1000F000523465347634523420344F346E342034E4
:1001000049346E34633420342034533465347434C9
:10011000423472346934673468347434203420349F
:1001200043346F346E34743420342034203420341B
:10013000593465347334203420344E346F342034D1
:100140002034523465347334653474343F3420348D
:10015000443465346634613475346C3474343F34FB
:1001600046346F346334753473344F3475347434B7
:1001700046346F34633475347334203449346E3408
:10020000A600030EA7000B1930298B182029270EF2
:100210008300A60E260E09006400810183160313D5
:1002200088308100831286140614A50183160313F7
:1002300019309900243098008312903098000800FB
:100240008B100C30A000A00B232906180729AD3015
:10025000810020308B000230A5000830A000072963
:100260000B1125194329A00803193C29060CA10CE0
:10027000A003AD3081000729061C59290130A500D3
:100280002108A2005929A5195929A00803195129A3
:10029000A30C031C861003188614A003B53081003C
:1002A00007290000000000008614A515A830810071
:1002B000072900308B000130A50507296400A80B31
:1002C0006E29A90BA82C0130AA06031D6929071461
:1002D0006A2907100030A8001830A9003030050541
:1002E000B1003202031D80210C300505B9003A022D
:1002F000031DAA213108B2003908BA00D629080026
:1003000032083106303C0319D429310DB206B21E31
:100310009A2941189C29AD08031D9829AE08031D90
:1003200097292B08AD002C08AE00AD080319AE03C9
:10033000AD03080041188B29AD0A0319AE0A2B083A
:100340002D02031D08002C082E02031D0800AD011C
:10035000AE0108003A0839060C3C0319D429390DBE
:10036000BA06BA1DC4294218C629B508031DC229F8
:10037000B608031DC1293308B5003408B600B50816
:100380000319B603B50308004218B529B50A0319C5
:10039000B60A33083502031D080034083602031D6F
:1003A0000800B501B6010800BB0A08006400050892
:1003B000033946050319032AC3080319032AC5088C
:1003C0000319032A87118716FF30C70000000000B9
:1003D00000000000000000000000000000006400B9
:1003E000C70BE6298712FF30C7000000000000009D
:1003F0000000000000000000000000006400C70BC7
:10040000F529C50308008715C301080087145E217C
:100410008C1E072A9818122A181D142A181218164A
:100420001A080800181218161A08A20087100800E7
:10043000A3005E210C1E192A2308990007115E21D2
:100440000C1E1F2A07150800633084001030DC00E2
:10045000062222088000840ADC0B282A5708013C67
:10046000031D492AC308031D492A73220830DC00F2
:1004700063308400640000086122840ADC0B3A2A9D
:100480008B220830DC00640000086122840ADC0B47
:10049000432A40242E2C4D22552ADB000830DB0253
:1004A0007322562ADB000830DB028B220830DC0086
:1004B00000308A005B0807206122DB0ADC0B582A27
:1004C0000800A3005E21A518622A86100630A50048
:1004D0000000B5308100A0308B000830A0005E2104
:1004E000A5186F2A0800FE3061224830612AFE30CC
:1004F0006122993061225E08832AFE3061225030E9
:1005000061225F08832A0310DA00DA0DDA0DDA07B8
:10051000DA0D5A0D612AFE30612247306122013026
:1005200061220230612AFE306122473061220830A8
:1005300061220130612AFF223F08B3003E08B40067
:10054000FF223F08AB003E08AC00AA22523018221E
:1005500040242E2C8312031700308D002B088C00B2
:10056000E2228312031701308D002C088C00E22256
:100570008312031702308D0033088C00E2228312AD
:10058000031703308D0034088C00E22A831203170E
:1005900004308D0041088C00E22A831203170530D5
:1005A0008D0042088C00E22A8312031706308D006A
:1005B0005E088C00E22A8312031707308D005F0863
:1005C0008C00E22A6400831603130D1683120313B2
:1005D0000D128B130B17831603178C130C15553044
:1005E0008D00AA308D008C1463000C118316031348
:1005F0000D12831203130D120B138B1708006330B7
:100600008400A401BF01BE01A408031D152B06220E
:100610002208203C0319042B22080D3C0319042B4B
:1006200022088000A40A840A072B84030030BC003F
:100630000130BD003F23A40B1E2B080084030030B3
:10064000BC000A30BD003F23A40B272B0800840305
:100650000030BC006430BD003F23A40B302B0800E9
:1006600084030330BC00E830BD003F23A40B392BCA
:10067000080084032730BC001030BD003F2B2F3012
:100680000002C000C00B452B08003D08BF0703183F
:10069000BE0A3C08BE07422B3B08BD00BC01BC2380
:1006A000203018224108303E1822203018224208FB
:1006B000303E1822203018220508BD00BC01BC23A2
:1006C0004024BB012E2C2D08AF002E08B0003508A9
:1006D000B7003608B8003708BD003808BC007923D9
:1006E000093018222F08BD003008BC0079234024AF
:1006F0002E2C2B301822AE2BFF223F08C100C62221
:10070000443018223F08303E182240242E2CFF226D
:100710003F08C200CD22523018223F08303E182236
:1007200040242E2CFF223F08B5003E08B600FF22D1
:100730003F08AD003E08AE005330182240242E2C56
:100740003408BC003308BD00AE23203018222C082A
:10075000BC002B08BD00AE2340242E2C2730BE0049
:100760001030BF00CD23400818220330BE00E8300F
:10077000BF00CD23400818220030BE006430BF0007
:10078000CD23400818220030BE000A30BF00CD2320
:10079000400818223D08303E182A2F30C000C00AF9
:1007A0003F08BD023E08031C013EBC020318CF2BCC
:1007B0003F08BD073E080318013EBC07080083122E
:1007C00003138501831606309F00FF308500FD303E
:1007D0008600C0308700831203130712071400300D
:1007E000AA00A8001830A9008714071587158712DA
:1007F00030300505B2000C300505BA00C501C30153
:100800000830C8000130C6000C21442400308B00A1
:10081000FF30D000CF00CE00CD00CC00CB00CA000E
:10082000C900D100D500D400D300D200D6000130D9
:10083000D7000030D800D900C830C625C830C6253A
:1008400077227D221630DC0007308A005C08163CD7
:10085000C0276122DC0B242C08304B2206220730F3
:100860008A00DA015A08D727FF3903192E2C2202F1
:1008700003193C2CDA0A322C07308A005A08E12F7F
:100880000D3018220A30182A640083120317003032
:100890008D00831603178C130C14831203170C0896
:1008A000AB0001308D00831603178C130C148312D8
:1008B00003170C08AC0002308D00831603178C134D
:1008C0000C14831203170C08B30003308D00831639
:1008D00003178C130C14831203170C08B400043094
:1008E0008D00831603178C130C14831203170C0846
:1008F000C10005308D00831603178C130C1483126E
:1009000003170C08C20006308D00831603178C13E2
:100910000C14831203170C08DE0007308D008316B9
:1009200003178C130C14831203170C08DF00031336
:10093000BB013308B5003408B6000310B60CB50C83
:100940002B08AD002C08AE000310AE0CAD0C080057
:1009500064004F08D0004E08CF004D08CE004C0870
:10096000CD004B08CC004A08CB004908CA00060855
:10097000C039C90050084F044E044D044C044B04C8
:100980004A044904D100C0390319112D5708013C0C
:10099000031D222D3230C4005108C03C0319EE2C37
:1009A0005208530454045504DA00DA1F0A2D5A1F62
:1009B000042D48080319DE2CC803002D5408D50067
:1009C0005308D4005208D3005108D2004030C80068
:1009D0000130C400D11F072D511F012DFF30D00061
:1009E000CF00CE00CD00CC00CB00CA00C900D100A2
:1009F000D500D400D300D2000830C8000030C500B4
:100A00006E29C308031D002D0230C6000C2DC3083B
:100A1000031D002D0130C6004408C5000130C3008D
:100A2000002D64005708023C0319002D0230D70046
:100A30000030D800D9001830522220304D22510801
:100A4000D600002D6400560851020319002DD60867
:100A5000031D312D5108C03A031D002D5108D60049
:100A6000002D5108D600511F5E2DD11F382DEE2CC0
:100A70005808013C0319B32D0130D80007308A0013
:100A80005908EA2F640058305222682D640058300B
:100A90005222702D6400803052227B2D6400803001
:100AA0005222892D640098305222A0304D22002D10
:100AB000640098305222A8304D22002D58080319A6
:100AC000AD2D07308A005908F22F0130C106C62229
:100AD0006030411868304D22002D0130C206CD2211
:100AE0007030421878304D22002D5E080A3C031900
:100AF000DE01DE0AD42288304D2293225E082F3E8A
:100B000061227722002D5F080A3C0319DF01DF0A0A
:100B1000DB2290304D2293225F082F3E61227D22FE
:100B2000002DDF2B0301AB00B3002030AC00B4007C
:100B3000AA220301C100C200C622CD220630DE0077
:100B4000DF00D422DB2277227D22B32D0030D800B3
:100B50000130D70008304B22002D5908013ED90042
:100B6000073C0319D9010310D8015908DA00DA0D3E
:100B7000DA0DDA0D20305A074D2218305222002D9E
:100B80007C30E1006400E10BC22D0800E200C025CA
:060B9000E20BC72D080076
:100F80008207FE344E34013404340E3415340434F4
:100F90000434043404340034FE344E340234043453
:100FA00004340434043415340E3404340034820719
:100FB00051345634763453345234483471344C34CA
:100FC00000348207632B7C2B872B922B9B2AA02B30
:100FD0004C2B242A8207422D462D4A2D4E2D522D70
:100FE000582DA62D8207652D6D2D752D832D912DE4
:040FF000922DA62D6B
:02400E00713F00
:104200000000200000002000000000000600060062
:00000001FF
